:1000000000308A003C280000831A0A28A500030E4D
:10001000A6000F288312A500030EA600A6140A0846
:10002000AD008A018313A50E0408A7002008A800CC
:100030002108A9002208AA002308AB002408AC006C
:1000400083128C308400001C27280C1842282708B3
:1000500084002808A0002908A1002A08A2002B0873
:10006000A3002C08A4002D088A00260E830083120A
:10007000250EA61883160900FF2383169000003072
:100080008A0098290030AE02031C0130AF02013013
:10009000031C0230B0020030031C0130B102B10871
:1000A000031D67283008003C031C67284030AE075A
:1000B000423003184330AF070F3003181030B00739
:1000C000003003180130B107B20A0319B30A0C104B
:1000D0008A112728B1010F30B0004230AF00403004
:1000E000AE000530900083160C148312DB29BC018E
:1000F0003C08033C031C8E283D30C1003C084107EE
:1001000084003C083B07C300430883169B009C13F4
:100110001C141A0880008312BC0A78283D08A0002D
:100120003E08A1003F08A2004008A300E3298E304A
:10013000A0003B08A0023C08A2003D08A100A217B5
:10014000A0080319AE280310A208031DAA28A108BD
:100150000319AE28A20CA10CA00BA328BC1FB52824
:10016000A109A209A10A0319A20AEC293C308400C2
:1001700000080319CC280130A100BF30A0006400A2
:10018000A00BBF28A10BBD284A30A000A00BC62899
:1001900000006400800BBB2800343A15B501013023
:1001A000B400B508031DF2283408033C031CF228F0
:1001B0008316051083120514831605118312051585
:1001C000C830BC00B62083160510831205108316B4
:1001D000051183120511C830BC00B620B40A0319FA
:1001E000B50AD1280430BB00FA30BC00B620BB0BE6
:1001F000F428B301B2013A1D972983160C14831217
:1002000036083202031D08293708330203191A2958
:100210003308B7003208B60083160511831205159E
:10022000C830BC00B6208316051183120511C830F2
:10023000BC00B620831605168312051A9629FA30DB
:10024000BC00B62083160C1083123308B9003208A4
:10025000B8003A113908BC003808BB008E30A00045
:100260003C08A1003B08A200A301A108031D4229EC
:100270002208A100A2010830A002A108031D422902
:10028000A0014A290310A11B4929A20DA10DA00319
:100290004229A1132008BB002108BC002208BD0090
:1002A0002308BE000130BF003E08C3003D08C20065
:1002B0003C08C1003B08C000C4014408033C031CC7
:1002C000852944083F07C5004030C600440846075A
:1002D00084000008C700450883169B008312470866
:1002E00083169A001C1583120B08A0008B1383162B
:1002F00055309D00AA309D009C149C187D291C112E
:10030000831220088B04C40A5D290A30BC00B62081
:100310008316051083120514C830BC00B62083165E
:10032000051083120510B301B2019729FB280A2A90
:1003300003081F3983003F30A0002130840083135D
:100340008001840AA00BA029A00184011F3083052D
:100350001F1383161F109F101F119F110730831248
:100360009900B201B301B401B5010B30B800B90175
:100370003A10BA103A111F1383161F109F101F1145
:100380009F1183121F1083160108C7390838810096
:100390000730831299008316050885006400023037
:1003A0008312A000A00BD229D52919088C1183161D
:1003B000990183126A28C0308B0483160C10013017
:1003C0008312BB0077282308BE002208BD00210845
:1003D000BC002008BB0097282208B9002108B800FB
:1003E000B808031DF629B9080319FB29380FFE299F
:1003F000B908031DFE29B9010B30B8008316051694
:100400008312051A0A2A3A180A2A3A146430BC00E0
:10041000B620CD28831605168312051A2B2ABA1882
:100420002B2AFA30BC00B620B301B201BA148316ED
:1004300085108312851483160C140510831205147D
:100440000230BB009630BC00B620BB0B222A8316BC
:1004500005108312051038083202031D5D2A390881
:100460003302031D5D2ABA1C5D2ABA1083160C10D4
:100470008312B301B201B701B6018316851083124E
:100480008510B5010130B400B508031D5D2A34089C
:100490000F3C031C5D2A8316051083120514C83017
:1004A000BC00B6208316051083120510C830BC00AE
:1004B000B620B40A0319B50A442A36083202031DCD
:1004C000652A370833020319772A3308B700320840
:1004D000B6008316051183120515C830BC00B6207E
:1004E0008316051183120511C830BC00B6200A2AF4
:0204F0006300A7
:02400E0004317B
:00000001FF
